:0A000000762C000000000000302DF7
:10000A008316A503A5032508003C03181128A50398
:10001A0000000000000008280000000000000000A6
:04002A0000000800CA
:10002E007408F8027508031C750FF9027608031C94
:10003E00760FFA027708031C770FFB02F30D0730D9
:10004E00FC00730DF80DF90DFA0DFB0D7408731C01
:10005E003E28F8027508031C750FF9027608031C7A
:10006E00760FFA027708031C770FFB024B28F8076E
:10007E0075080318750FF90776080318760FFA0737
:10008E0077080318770FFB07F30DFC0B2828720D6A
:10009E00F80DF90DFA0DFB0D7408731C6428F802A7
:1000AE007508031C750FF9027608031C760FFA0209
:1000BE007708031C770FFB027128F80775080318E1
:1000CE00750FF90776080318760FFA0777080318E5
:1000DE00770FFB07F20D0730FC00720DF80DF90DCE
:1000EE00FA0DFB0D7408721C8A28F8027508031CA1
:1000FE00750FF9027608031C760FFA027708031CB7
:10010E00770FFB029728F80775080318750FF90784
:10011E0076080318760FFA0777080318770FFB0790
:10012E00F20DFC0B7428710DF80DF90DFA0DFB0D87
:10013E007408721CB028F8027508031C750FF902BA
:10014E007608031C760FFA027708031C770FFB0262
:10015E00BD28F80775080318750FF90776080318F8
:10016E00760FFA0777080318770FFB07F10D0730A4
:10017E00FC00710DF80DF90DFA0DFB0D7408711CD4
:10018E00D628F8027508031C750FF9027608031CB1
:10019E00760FFA027708031C770FFB02E328F807A5
:1001AE0075080318750FF90776080318760FFA0706
:1001BE0077080318770FFB07F10DFC0BC028700DA5
:1001CE00F80DF90DFA0DFB0D7408711CFC28F802E0
:1001DE007508031C750FF9027608031C760FFA02D8
:1001EE007708031C770FFB020929F8077508031817
:1001FE00750FF90776080318760FFA0777080318B4
:10020E00770FFB07F00D0730FC00700DF80DF90DA0
:10021E00FA0DFB0D7408701C2229F8027508031CD8
:10022E00750FF9027608031C760FFA027708031C85
:10023E00770FFB022F29F80775080318750FF907BA
:10024E0076080318760FFA0777080318770FFB075F
:10025E00F00DFC0B0C29701842297408F80775086C
:10026E000318750FF90776080318760FFA07770843
:08027E000318770FFB070800CD
:10028600FB09FA09F909F809F80A0319F90A031921
:08029600FA0A0319FB0A080033
:10029E0083120313F801F9011030FC00710DF80DF3
:1002AE00F90D7408F8027508031C750FF90203188E
:1002BE0067297408F80775080318750FF9070310F6
:0A02CE00F00DF10DFC0B552908009E
:0C02D800831254088A00530882000800BA
:1002E40001308316A40083125608EF0659088400CF
:1002F4005608003A031981295008800483295508B7
:10030400800557088316A50005208312EF0983167C
:1003140024080319A629240883126F05F000031D7D
:100324009629500880049829550880058316A40D41
:1003340024100230831257028316A5000520000002
:10034400000000000000892983125608003A0319AE
:10035400AE2955088005B029500880045708831633
:06036400A50005200800C1
:0C036A000E30FD00FD0BB729000008005C
:1003760040308312F0001F30F100F201F301080053
:1003860083126F08F2007208F000F20A7008840007
:1003960000080319CF29C6296F087202F000013040
:0A03A600F002F101031CF10308004E
:1003B00083120313F8010830FC00700DF80D740867
:1003C000F8020318E529F8070310F00DFC0BDD29EE
:0203D000080023
:1003D200831203132230FC00F801F901FA01FB0138
:1003E200FC0303191F2A0310FB0CFA0CF90CF80C7E
:1003F200F30CF20CF10CF00C031CF129FC030319B1
:10040200112A7408F80775080318750FF90776089A
:100412000318760FFA0777080318770FFB07F529F9
:100422007408F80775080318750FF907760803189A
:0E043200760FFA0777080318770FFB0708000C
:1004400083120313FC01F71BFC0AFD01FB01FA01F7
:10045000F901F80173087204710470040319B42AD5
:1004600073087706D800D81BFD09F71F422AF40944
:10047000F509F609F709F40A0319F50A0319F60A4A
:100480000319F70AF31F4F2AF009F109F209F309DA
:10049000F00A0319F10A0319F20A0319F30A73089F
:1004A0007704D800D81B702A1720FC1B8D2AFD1F4B
:1004B000B42AF009F109F209F309F00A0319F10A63
:1004C0000319F20A0319F30AF809F909FA09FB09F1
:1004D000F80A0319F90A0319FA0A0319FB0AB42ADC
:1004E000F71F872AF31B812A7308FB007208FA00A2
:1004F0007108F9007008F800F301F201F101F00150
:10050000572AF301F201F101F001F00A0034F30976
:10051000F209F109F009FC17542AF80A0319F90A3B
:100520000319FA0A0319FB0A74087802031D572AF3
:1005300075087902031D572A76087A02031D572A87
:1005400077087B02031D572AFB01FA01F901F80124
:10055000F00A0319F10A0319F20A0319F30AF31F47
:10056000572AD8015816FF34D8017C1CB82A4321D9
:04057000003E080041
:1005740083126108F2007208F100F20A6208F000C6
:10058400E20A700884000008F00071088400700812
:1005940080007108840000080319D12ABD2A61086B
:0405A400F00008005B
:1005A8006C218A110A128000840AD30A0319D40A1A
:0805B800F003031DD42A080022
:1005C000F03083129F05F03083169F0483129F172B
:1005D0006108F000F00D7010F00D701070089F04AD
:1005E0001F14B5219F149F1CF72A0000F32A1F1027
:1005F0001E08F100F00183161E08F0040030F1041B
:020600000800F0
:1006020083126108EF00C3217008E300E20162086F
:10061200610784000008EF0072218312E20A803031
:100622006206F000803063067002031C082B08008B
:100632000A308312EF0072210D308312EF00722113
:020642000800AE
:1006440083126108D9006208F0000130F2007008DA
:100654000319302BF20D7210FF3E2A2B7208DA00B8
:100664007209DE006308F1000130F000710803191B
:100674003F2BF00D7010FF3E392B7008D000F009AD
:100684007008D50080306107840072088004700807
:100694008005D60168080319502BD609841356081F
:1006A400003A0319582B550880055A2B500880042A
:1006B400BB21E830F4000330F500F601F701E9212D
:1006C4007008E9007108EA007208EB007308EC0096
:1006D4006408F0006508F1006608F2006708F3009A
:1006E400F00DF10DF20DF30D7010F00DF10DF20D92
:1006F400F30D70100A30F400F501F601F701E92159
:1007040070088316A0007108A1007208A200730883
:10071400A3007008F4007108F5007208F60073086D
:10072400F70083126908F0006A08F1006B08F20010
:100734006C08F30020227008ED007108EE007108C7
:10074400F400F501740875040319AB2B0230F000B2
:1007540008006D08D70083162008F4002108F5006E
:100764002208F6002308F70083126908F0006A08DB
:10077400F1006B08F2006C08F30020227808F00006
:100784007908F1007A08F2007B08F3007008E900A8
:100794007108EA007208EB007308EC008316200865
:1007A400F5002108F6002208F7002308F800F80CE9
:1007B400F70CF60CF50CF813781BF8178030780654
:1007C400F400803073067402031DF22B7208770262
:1007D400031DF22B71087602031DF22B70087502BB
:1007E4000318F62B8312D70A83125708F100F10C71
:1007F400F1137108D200073071020318042C013080
:08080400F0000800F0010800FB
:10080C008312E301033063020318132C630862079D
:10081C00840020308000E30A082C630862078400FF
:10082C008001E30363086207E4000A30F400610806
:10083C00F000D8217808F0003030F007640884000C
:10084C00700880000A30F4006108F000D8217008AC
:10085C00E1007008003A031D342C362CE303182CED
:02086C00080082
:10086E008312E401053064020318442C6408630704
:10087E00840020308000E40A392C64086307840069
:10088E008001E40364086307E5000A30F400F50113
:10089E006108F0006208F1004F217808F000790835
:1008AE00F1003030F00765088400700880000A30CF
:1008BE00F400F5016108F0006208F1004F217008A4
:1008CE00E1007108E20000307106031D702C00304B
:0E08DE007006031D732C752CE403492C0800D2
:1008EC0090258316960183161D308500FF308312E8
:1008FC0099002830831695001C309F008C018312C0
:10090C008C01831681018312CF018512CE01053033
:10091C00E100003005180130E2000030851801308C
:10092C00E3008030E4002530E500E601E701E80152
:10093C0022237008D1007008003C0318B62C20301C
:10094C0085060630FB001330FC00AD30FD00FD0BBE
:10095C00AD2CFC0BAD2CFB0BAD2C00000000A52C22
:10096C00192383123708E1002130E200BA22700803
:10097C00B7007008E100012319230B30FB0026306F
:10098C00FC005D30FD00FD0BC92CFC0BC92CFB0BD6
:10099C00C92C00000000831285169F01FF308F00C8
:1009AC009B308E00113090000C1083160C14C0304C
:1009BC008B000D3083129F0083120330E100E02284
:1009CC0070088312DC007108DD007008F2007108F9
:1009DC00F300F30CF20CF313F30CF20CF313720898
:1009EC00DB00851D292D5C08E1005D08E20037085D
:1009FC00E30037243708E10001230930EF007221AE
:100A0C0083125B08E1003708E20006243708E10096
:100A1C0001230930EF00722183124F08E1003708DF
:100A2C00E20006243708E10001230230FB00043009
:100A3C00FC00BA30FD00FD0B212DFC0B212DFB0B16
:0A0A4C00212D00001923E22C2A2DB1
:100A6000FF00030E8301DF000A08E0008A0170081E
:100A7000A0000C1C592D4E08003A031D432D5B08A5
:100A8000CF0085168512CE0A4E084F06031D492D4C
:100A90008516851D522DEC308F0078308E00213068
:100AA0009000582DFF308F009B308E001130900049
:100AB0000C102008F00060088A005F0E8300FF0E13
:040AC0007F0E09009C
:100B2000213084002D308312F0006230D300053074
:060B3000D400D4220800ED
:100AC40054346534733474342034503457344D34CE
:100AD4002034613476346534633420343134323430
:0C0AE40046343634383433340A340034DD
:020AF000383498
:100AF20030343134323433343434353436343734B8
:100B020038343934303431343234333434343534A3
:0C0B120036343734383439343034003491
:02400E00C400EC
:00000001FF
